:030000000219FDE5
:03000B000200A848
:03002B0002015D72
:03005B000202DCC2
:030073000202C2C4
:1000800002030406080C10182030406080040608A3
:100090000C10182030406080A0C000070F1F3F05E3
:1000A000050D050205030302C2AFC0D0C0E0206207
:1000B00017E5256002E473E525F4F58A758B00D217
:1000C00062D0E0D0D0D2AF3285268AC262E526F473
:1000D000602F758B00D0E0D0D0C293C295C297D26A
:1000E000AF32C293C295C297206E0C206609740E7F
:1000F000D5E0FDE57E4290758B00D0E0D0D0D2AF48
:1001000032758A00C28DD26201F701B730680520CE
:100110006602D29301B7306805206602D29501B716
:10012000306805206602D29701B7C29230680A2073
:100130006607740CD5E0FDD29301B7C29430680A0B
:10014000206607740CD5E0FDD29501B7C2963068E1
:100150000A206607740CD5E0FDD29701B7C2AFC282
:10016000AD53E6EFC0D0C0E0D2D3D2AFC2CEE52AC5
:100170006007207449152A21BE7800790020742E6A
:10018000E580307E01F430E30278FF53DACF207E41
:100190000343DA20307E0343DA10C2D8C271E5800F
:1001A000307E01F430E30279FFC3E89970CB30610F
:1001B00003752A18207403752A18885FD27020747A
:1001C0000DE52B6004152B21CE43DA01C2D8207037
:1001D000024130A85F206102C270207431C3E894EC
:1001E000F0400374F0F8E8C4540F28F87984B7039A
:1001F00002410EC313C3138721200802C313200A30
:1002000006C3C898F8410E28F8500374FFF8C3E8F5
:1002100095685003E568F88822E52D54066011E5DD
:1002200033C313C31324062522F52250037522FF7E
:10023000852224A824C3E52495644002A864882567
:10024000E56970024174C3E8AA699A5003E8FAE4C8
:10025000F9EAC333FBE56BF45B29400D256AF8E549
:100260006A6002156A400B41740AC3E56A9A50023B
:10027000056A78FF8826C3E52594404002D26420B1
:10028000CF0AD0E0D0D043E610D2AD32C2CF053A8B
:100290007801E52A6005307402152AC3E55F9401F0
:1002A000400575620041B8756300756C00E5622415
:1002B00001F56250037562FFD0E0D0D043E610D262
:1002C000AD32C2AFC0D053E67FC260759100855693
:1002D00094855795759104D0D0D2AF32C2AF53E612
:1002E000EFC2ADC0D0C0E0C0F0D2D3D2AFA8FBA95E
:1002F000FCC2D8307102614353DACF207E0343DA67
:1003000010307E0343DA20D271E580307E01F42084
:10031000E302611A88278928A17053DACF207E036F
:1003200043DA20307E0343DA10C2D8C2713074023F
:10033000A15C7800E580307E01F430E302A15C88A6
:100340005FA14453DACF207E0343DA20307E03439B
:10035000DA10C271206102811C53DACF207E034380
:10036000DA10307E0343DA20C2D8D271885A895B12
:10037000C3E89558F8E99559F97B007E087A00C3DF
:10038000E8948CE994005005755E00810E88217810
:10039000A2E6A8216055C3E894C8E994005008E497
:1003A000D2E4FB7A0A61E9C3E89468E99401500851
:1003B000E4D2E3FB7A0F61E9C3E894D0E9940250F8
:1003C00008E4D2E2FB7A1E61E9C3E894A0E994054F
:1003D0005008E4D2E1FB7A3C61E9C3E89498E994DF
:1003E000085008E4D2E0FB7A787E00C3E8955CFC14
:1003F000E9955DFD30E70AECF42401FCEDF43400EE
:10040000FD755E00C3EC9AED9E5003755E01885C3D
:10041000895D855A58855B597802A144C3E89527C0
:10042000F8E99528F9307C02A128307B02A1283018
:100430007A02A121207502813FE9FDE8FC815EE995
:10044000C313F9E813F8307902A121E9C313F9E8DD
:1004500013F8307802A121E9C313FDE813FC2061F1
:100460002CC3EC941CED940240028175ED701EC308
:0E047000EC94C850180529E52970021529C31F
:10047E00E529940A5002A15C755F00D270A15CE57B
:10048E0029600215297888E6F97400207F0878968D
:10049E00B90302789EE624FAFEE43400FFC3EC9E14
:1004AE00FCED9FFD9208B90310A2085007207609B3
:1004BE00D27681C7307602C276A2085016B9030DE5
:1004CE00ECF42401FCEDF43400FD0204E178007933
:1004DE0000A128B90315EC33FCED33FDC3EC940AEF
:1004EE00FCED9400FD50047C007D00C3EC94FFED08
:1004FE009400400678FF7900A128EC8575F0A4C51C
:10050E00F0A2F733F87900400302054478FF790032
:10051E00020544E9C313F9E813F8307C0EE96002D2
:10052E0078FFC3E81338F8E43400F9C3E894FFE920
:10053E009400400278FF885FD270206102A15C7443
:10054E001FF4552F4BF52FC274EB7002D274752A1F
:10055E0018307403752A0A306102A1702074035397
:10056E00DAFE207403752B06D0F0D0E0D0D0D2ADD9
:10057E0043E6103279010205A079030205A0790A3B
:10058E000205A0791E0205A079640205A079C802B1
:10059E0005A07817E4D5E0FDD8FAD9F6227A147BB7
:1005AE00780205C77A107B8C0205C77A0D7BB402E0
:1005BE0005C77A0B7BC80205C77902B27DE4C294E7
:1005CE00D5E0FDD295D5E0FDC295D5E0FDD294D50E
:1005DE00E0FDD293E576D5E0FDC2937496D5E0FDAD
:1005EE00D9D9EAF8D5E0FDD8FBDBCEC29422C37C84
:1005FE00007D0075F00005F0EA33FAEB33FB50F6A0
:10060E00EB13FBEA13FAC3E9FFE8FEE89AF8E99B5D
:10061E00F95004EFF9EEF8B3EC33FCED33FDD5F001
:10062E00DFEDF9ECF822E889F08A20D2D4F8A9F0AF
:10063E007B0030F70B7BFFF42401F8E9F43400F96A
:10064E00E88520F0A4ADF0F8E98520F0A4AFF0FE27
:10065E00ED2EF974003FFA7C04C3EA13FAE913F99C
:10066E00E813F8DCF48BF030F70AE8F42401F8E92B
:10067E00F43400F9E889F0C2D4F8A9F02222C3E5D7
:10068E004113F9E54013F8C3E54598F8E54699F9A5
:10069E00500CC3E89480E994FF40160206C3C3E8E9
:1006AE00947FE9940050030206C3787F7900020616
:1006BE00C3788079FF884A894B22E54A2547F8E5B9
:1006CE004B3548F9854B20E4300701F43549FA30B3
:1006DE00E709C3EA94F04015020701C3EA940F50EC
:1006EE000302070178FF79FF7A0F0207017800797C
:1006FE00007AF0C3E5249564500AC3740195245022
:10070E000B02071FE54B20E70E02071FE54B30E7F4
:10071E0006884789488A492278A4E6FAC3E54A330F
:10072E00F8E54B33F9D134E930E70BC3E89480E9AF
:10073E0094FF4013E159C3E8947FE994005002E11D
:10074E0059787F7900E159788079FFE820E715C361
:10075E00E52398F84009C3E8940140030207807826
:10076E0001020780E8F424012523F84003020780E4
:10077E0078FF884C2278A5E6FAA848A949D134E931
:10078E0030E70CC3E89401E994FF40160207B4C3A6
:10079E00E894FFE9940050030207B478FF79000251
:1007AE0007B4780179FFE920E715C3E54C98F840C6
:1007BE0009C3E8940140030207DB78010207DBE876
:1007CE00F42401254CF840030207DB78FF8824222D
:1007DE0078FFC26420693D206A12D264C3E5419459
:1007EE000A4009C3E52594405002C26479A1E7602E
:1007FE0023E541601F74FF8541F0848539F0306A2E
:10080E000375F005A4F8C5F0600278FFC3E895679C
:10081E005002A867886622C3E5409440E5419401E2
:10082E00E5665003140136046002F5662202083EA6
:10083E002275E890227883E6FFE5E820ECF7A8BD64
:10084E00A9BE0573C3E57394084052757300E9FAA7
:10085E0079A0E76044EA7007E574601B020879C36B
:0F086E00E895746010E5745006600C140208855C
:10087D000460F9020885E574F574C394A8401B75EE
:10088D0064C0C394054013756480C39405400B7513
:10089D006440C39405400375640075BB0122E56493
:1008AD00F460020564E573B4070375BB1E22743250
:1008BD0079A687F0A4C5F0A2F733F8C3E895644094
:1008CD0002A8648822882488258826886722754096
:1008DD00007541F022C2AF75C820A8CCA9CDAA3AA7
:1008ED0030CF010A75C824D2AFAB3BAC3C883B89F5
:1008FD003CC3E89BF8E99C206908F930670221F7B1
:10090D002154AD3D8A3DF9EA9DFA600478FF79FFE7
:10091D00AE3EAF3F8B3E8C3FC3EC9FFCC3E99CF5D5
:10092D0042A83BA93CC3E89EF8E99FF9C3E54113F2
:10093D00FBE54013FAE82AF540E93BF54150067511
:10094D0040FF7541FF219EAA40AB41AC40AD417EB9
:10095D00047F02C3EB940440021E1FC3EB940840B6
:10096D00021E1FC3ED13FDEC13FCDEF7C3EA9CFA68
:10097D00EB9DFBEF6009C3E913F9E813F8DFF7EA24
:10098D0028FAEB39FB8A408B4150067BFF8B408B5D
:10099D0041C3EB94025002D2673069047F0321C931
:1009AD007892E6FFC3E537948240110FC3E5379483
:1009BD00A040010FC3EF940640027F057E06E5417E
:1009CD00C4540FF9E541C454F0F8E540C4540F2860
:1009DD00F8C3E89EFAE99400FB4009C3EA9402EBE0
:1009ED00940050047A02E4FB4143AA40AB41EBC4AE
:1009FD00FEEAC4540F4EFCC3EA9CFAEB9400FBC311
:100A0D00E813C313F8EA28FAEB3400FB8A408B4154
:100A1D00C3EB94024002C2677806EBC4FE7B00EA8A
:100A2D00C4540F4EFAC3EA98FA4005C3940250021B
:100A3D007A027892E6FF3060024143855256855323
:100A4D0057D26043E680C3E49AF8E49BF93067021D
:100A5D0041DDE8FAE9FBD3E913FDE813FC8852897F
:100A6D0053C3EF94036038EF20E00DE82CF8E93D17
:100A7D00F9ECFAEDFB020A98E828F8E939F9C3E830
:100A8D002402F8E93400F97AFE7BFFC3EF940340AA
:100A9D000E8A548B55884E894F8C508D516111881B
:100AAD005489558A4E8B4F8C508D51306920C3E53A
:100ABD003394034019E542A2E713F8E555F42401F8
:100ACD0038400B20E7087554FFF42401F5556111EA
:100ADD00E8FAD3E813FC8852C3EF94036020EF20AB
:100AED00E007E82CF8ECFA41FDE8282402F87AFE3C
:100AFD00C3EF940340088A54884E8C50611188547A
:100B0D008A4E8C50E56BC3335002646BF56B3060CD
:100B1D0002611B753402D26043E680E52D540660F8
:100B2D0026A840A941C3E913F9E813F8C2AF53E66B
:100B3D007F759100C3E498F594E499F5957591044A
:100B4D00D26043E680D2AF22D26575440075200095
:100B5D00306B03752040020B74D26575440075200F
:100B6D0040306B03752000D2AF7801206722E52D50
:100B7D0054066002C265C3E54194054013780294A2
:100B8D000540087803940540027806306902780A1A
:100B9D00206019E544601530690AC3E533940340BC
:100BAD0003D53406D2AFD26C814E7123D2AF000083
:100BBD00C2AF206726E541C3FB940F40027B0FEBCC
:100BCD00240530730123306A02742820620123F951
:100BDD003069027982E58BC39940B50544E59E7075
:100BED0005E59B020BF5E59A5440B520028138309E
:100BFD00690A08C3E8940A400108619D20650261F5
:100C0D0074C26553E67F7591003067107594007559
:100C1D0095FE759104D26043E6806174AE40AF419C
:100C2D00C3E49EF594E49FF595811FC3E5339402CB
:100C3D00500261743065026174D802814C619DC2AD
:100C4D006C53E67F75910085549485559575910487
:100C5D00854E56854F57D26043E680D2AFE52D5471
:0E0C6D00066008206A020533020C88306C0D08
:100C7B00206B0A2065071581158102152A22780041
:100C8B003064053065027801E53775F007A4F9E5A6
:100C9B00F028F5F0E9A2F013A2F113A2F213F53745
:100CAB00C394785003753778C3E53795384008D22D
:100CBB0066C293C295C29730600281C28550568539
:100CCB005157D26043E68022207D14C2AF75430298
:100CDB00C294D292D2AF759F33759E00020EB4C2EE
:100CEB00AF754302C294D296D2AF759F33759E00F7
:100CFB00020EB4307243207D20C2AF7543039001C6
:100D0B003B757E10C297C296306204D295A11CD25D
:100D1B0094D2AF759E23020EB4C2AF7543039001FC
:100D2B003B757E10C293C292306204D295A13CD225
:100D3B0094D2AF759E22020EB4207D17C2AF7543BD
:100D4B0003900116C297306202D295D2AF759E23E3
:100D5B00020EB4C2AF754303900116C29330620208
:100D6B00D295D2AF759E22020EB4207D11C2AF7503
:100D7B004304C292D296D2AF759E22020EB4C2AF7A
:100D8B00754304C296D292D2AF759E23020EB43035
:100D9B007249207D23C2AF75430590012A757E04ED
:100DAB00C295C294306204D293A1B8D292D2AF75DD
:100DBB009F33759E00020EB4C2AF75430590014C74
:100DCB00757E40C295C294306204D297A1DBD29655
:100DDB00D2AF759F33759E00020EB4207D1AC2AF41
:100DEB0075430590010CC295306202D293D2AF7558
:100DFB009F33759E00020EB4C2AF75430590012060
:100E0B00C2953062E8D297D2AF759F33759E0002C0
:100E1B000EB4207D11C2AF754306C296D294D2AFE9
:100E2B00759E23020EB4C2AF754306C292D294D202
:100E3B00AF759E22020EB4307242207D20C2AF7578
:100E4B00430190014C757E40C293C292306204D232
:100E5B0097C160D296D2AF759E22020EB4C2AF7507
:100E6B00430190012A757E04C297C296306204D268
:100E7B0093C180D292D2AF759E23C1B4207D16C28E
:100E8B00AF754301900120C293306202D297D2AF6B
:100E9B00759E22C1B4C2AF75430190010CC297304D
:100EAB006202D293D2AF759E23C2662290010A755D
:100EBB007E00C293C295C297C292C294C296C2627E
:100ECB0022788076FF0876FF0876FF0876FF087693
:100EDB000308760408760708760108760108760180
:100EEB00788C76010876FF0876FF0876FF0876FF88
:100EFB000876FF0876030876FF0876FF0876FF086A
:100F0B0076250876D00876FA0876FA0876040876FD
:100F1B00FF08760108760008767A0876FF087601D6
:100F2B00087601087600087603227887E6FFC272FE
:100F3B007888E6C394036008C27DE630E102D27D77
:100F4B00C27E7889E630E102D27EC3EF940260085C
:100F5B00758E01D273020F68758E00C27322788072
:100F6B00E6149000809378A4F67881E614900080C4
:100F7B009378A5F67886E61490008D9378A6F6788C
:100F8B009CE67538FF75390CB402067538A07539B7
:100F9B000AB4030675388275390578A3E6149000F8
:100FAB009A93F569D1B722227896E6FA7897E6FB01
:100FBB007888E6B40305C3EB940EFB307F047A000C
:100FCB007BFFC3EB9AFCC3948250027C8275750045
:100FDB000575EC8575F0A4C3E5F0947D40F222D243
:100FEB007FF1B31205917A007B007C10120587E527
:100FFB005F2AFA74003BFBDCF37C04C3EB13FBEAC4
:10100B0013FADCF7FEC27F120FB322E5EF20E603E3
:10101B007520000520903DFFE520146006901FFF12
:10102B001460009304600375EF1253D9BF7581C030
:10103B0043FF8012058275EF0243B203E5B324042C
:10104B0020E70DF521E5B120E0068521B343B10181
:10105B00120EB77580FF75A40075F1FE75D4F77588
:0E106B00900275A5FC75F2FC75D50075A0FD10
:1010790075A60275F30275D60075B0FF75A70175DF
:10108900F4FF75E241E4F8F6D8FD756B01120ECC58
:1010990012156C78988676753001C2AF12059B12CD
:1010A90005AB1205911205B21205911205B9120587
:1010B9009112168512059B12059B120596C2AF78EF
:1010C900FA79FA308307D9FBD8F7021C00120F35D9
:1010D900120F69120FB2120FB378988676120EB7F3
:1010E90075885075891275C82475910475D840752D
:1010F900A82275B80275E690759B80759D00759A52
:1011090080759C0075D10E75BC5875BB0175BA1FE9
:1011190075E880120582D2AF12083B53DACF207EE0
:101129000343DA20307E0343DA1043DA01C2D8C21E
:101139007112059BD2617B037A0CE55E70077A0C0C
:10114900DB030210C61205912070030210C6C2709B
:10115900E55FC3940240E1E52F541F856160F561A5
:10116900B560D5DAD5C26153DACF207E0343DA20E0
:10117900307E0343DA10C2D8C27178A2E67008D271
:1011890074E52F54E0F52FC27575290012059630C4
:101199007409C3E529940A4002D2751205877802B9
:1011A9003074027800C3E55F9840F0C2AF1205AB16
:1011B9001205AB1205ABD2AF12059B754D007888AD
:1011C900E6B4030241AC120587788CE6C39401505A
:1011D900030212ACE530C3940150030212AC20742F
:1011E90035C3E55F94FF50030212ACC2AF1205C0CC
:1011F900D2AF120596C3E55F940150EFC2AF120555
:10120900AB12058C1205ABD2AF120596C3E55F94FC
:10121900FF40E902170A7F05D27F120FB312059624
:10122900C2AFC27F120FB3AE5FC3E55F947FD2AF87
:10123900407B120582C2AF1205C0D2AFDFDA120FAE
:10124900EAC3EE94057897F612059B1215AE1216AD
:101259008D7F0AD27F120FB3120596C2AFC27F12D9
:101269000FB3AE5FC3E55F947FD2AF50E41205823E
:10127900C2AF1205AB12058C1205ABD2AFDFD41287
:101289000FEAEE24057896F612059B1215AE121692
:10129900BC120596120FB3C3E55F94FF500221E714
:1012A90002170AC3E55F954D4003855F4D12059608
:1012B90078017988E7B403027805C3E55F984002AD
:1012C90021C7C2AF1205C01205C01205C0D2AF12A4
:1012D900059B753000E4F531F5320531E531F470DF
:1012E900390532789AE67819146012783214600D4B
:1012F900787D14600878FA146003753200C3E5320A
:1013090098401715327531B478998676C2AF1205AF
:10131900C0D2AF7898867612059612058CE52A70A8
:101329000530740201C678012074027806C3E55FAE
:101339009840A77888E6C394036003120596E52AC6
:1013490070030210C6C2AF120EB7E4F522F523F5F9
:1013590024F525F526F56AD2AF7885E6C333F56815
:10136900E4F545F546F547F548F549F573F52CF5E6
:101379002DF53775730875BB1E12058212083FE5F6
:10138900E820ECFBA8BDA9BEE97001F88874120831
:101399004375730875BB1E7887E6FE7602120F3512
:1013A9007887EEF6C2AF7564FF1208BB85226485A3
:1013B9002265852266D2AF75220175240175250142
:1013C90075260185636C756D017888E6B40307C2DB
:1013D9007D307602D27DD268D269753300120E1D36
:1013E900120E421208DB1208E21208DB1208E2129E
:1013F90008DB02140BC2AF120F35D2AF757300753B
:10140900BB01120B6612068B120C89120CD312083F
:10141900E2120B55306D0312068C2067031207DEAA
:10142900306703120825120C89120CFE1208E21209
:101439000B66306D031206C8120C89120D7512085D
:10144900E2120B55306D03120726120C89120D9A00
:101459001208E2120B66306D03120783120C89120F
:0E1469000E1D1208E212083F120B55120C89DC
:10147700120E421208431208E2306932206B2F85A0
:10148700676485676585636C756D0179187A0CC328
:10149700E53399400CC269D26A8A357564FF021434
:1014A700B5C3E55F9401400302140B021532306A9D
:1014B7001B206B18E535147004C26A61FEF535C34D
:1014C700E55F9401400302140B021532753600C321
:1014D700E5627882985054307404E52A604D788824
:1014E700E6B40317207D05207607A102307602A116
:1014F70002206B07D26B856764814A78F0306B05F1
:101507008567647820C3E541985002810B306B1BD7
:10151700C26BC27D307602D27DD26A75351285677D
:1015270064810B0536E55F6002A135753600C2AFF1
:10153700120EB77887E6FE7602120F357887EEF639
:10154700E4F522F523F524F525F526F568C268D2DA
:10155700AF120582120EB7307409C3E53694054001
:101567000201C641DE901A0D78201215F0E520B46D
:101577005A0CA31215F0E520B4A50302158E120E1E
:10158700CC1215AE0215AD901A0378807B0A12159E
:10159700F0A308DBF9901A0F788C7B181215F0A3CB
:1015A70008DBF9901A2722C2AF12162F12160990DC
:1015B7001A00740E1215F5A374041215F5A374140A
:1015C7001215F5901A0378807B0A1215F4A308DB2D
:1015D700F9901A0F788C7B181215F4A308DBF9120F
:1015E7001642121620901A2722E493F622E6438F1A
:1015F70001538FFD75EF0275B7A575B7F1F0538FDE
:10160700FE22438F02438F0175EF0275B7A575B7A9
:10161700F1901A0DF0538FFC22901A0D745AB1F500
:10162700901A0E74A5B1F5227A3079D07820901AE5
:1016370040B1F0E520F709A3DAF7227A3079D090A4
:101647001A40E7B1F509A3DAF922AB77A878BB010D
:10165700027984BB02027985BB03027986BB040247
:101667007992BB05027987BB060279A3BB0702798A
:101677009CBB08027988BB09027989E8F7227C05B7
:1016870012059BDCFB22C2AF1205AB1205B2120595
:10169700B91205C012058C1205AB1205B21205B9B5
:1016A7001205C012058C1205AB1205B21205B9124C
:1016B70005C0D2AF22C2AF1205C01205B91205B2DA
:1016C7001205AB12058C1205C01205B91205B2122C
:1016D70005AB12058C1205C01205B91205B2120529
:1016E700ABD2AF22AE77AF78C2AF1205AB1205AB64
:1016F7001205AB12058CDEF21205C012058CDFF85D
:10170700D2AF22D18DD185D18575770175780175D5
:101717007900D1EB7C05AD5F12059BC3ED955F703A
:10172700F5C3E55F9401400AC3E55F94FF403202C9
:101737001746D151B1AED18DC2AF75EF12D185DC4D
:10174700D50579C3E5799403500280C6D18505781C
:10175700E5771490009F93F808C3E57898500280C6
:10176700AED185D1850577C3E577940A5002809C71
:0C177700120ECCB1AEC2AF75EF12D185DE
:0319FD00021016BF
:101A00000E0414FFFFFFFF0304070101015AA501A3
:101A1000FFFFFFFFFF03FFFFFF25D0FAFA04FF01DE
:081A2000007AFF01010003FF41
:101A4000235467794B4631323041485623202020B9
:101A500023424C48454C4923463331302320202033
:101A60002020202020202020202020202020202076
:101C0000C2AFC2D353D9BF7581C043B20343FF8073
:101C1000752438752503B1C975EF0275E24043F1AB
:101C20000853A4F775D400D2837DFA780379E67C53
:101C300010752200752300901DD67B0675249875BB
:101C400025013083028142208308D8FBD9F9DCF7D3
:101C500081B4308308D8FBD9F9DCF781B4B189E4C9
:101C600093A3C39A6004DDC381B4DBDBB17B600264
:101C7000812B7B08E493FAA3B15CDBF87A30B15C8A
:101C8000752200752300B17BEAFCEBFDC3ED94FEE9
:101C9000400EB17B8A278B28ED30E0048A828B834B
:101CA000B17B7AC270D8C3ED94FE601350CEBD00F4
:101CB00025EC60097520007521FF0200008100A855
:101CC00027A9280809D804D90281D3B17FEA89AAB3
:101CD000F281C50D81A0C3ED94035049EDA2E092BD
:101CE000007AC5C3E5829400E583941C50902000DF
:101CF00010438F02438F0175B7A575B7F1F030001F
:101D00001FA827A9280809438F01538FFDD804D99C
:101D100002A12089AAE275B7A575B7F1F0A3A10DBC
:101D2000538FFC817C7AC1BD030CE493A3FAB140CC
:101D3000DCF8B138817C817EAA22AB23B15CEBFA5E
:101D4000EA6222752608C3E52313F523E52213F57D
:101D50002250066323A0632201D526EAB1C9B1C986
:101D600075260AEAF4200102D283300102C283B14F
:101D7000C9C3134002C201D526EB22B17FEAFB2082
:101D80008302A17F308302A184752608AE24AF258B
:101D9000C3EF13FFEE13FEB1CDB1C9C3EA13308315
:101DA000024480FA30E703632201C3E52313F523DD
:101DB000E52213F52250066323A0632201D526D91C
:101DC000E52265236523F52222AE24AF250E0FDE22
:101DD000FEDFFCD20122424C48656C693437316326
:041DE000F3100601F5
:00000001FF
